:020000000C28CA
:10000800FE000308F1000408F2000A08F3006C2C53
:10001800192D83169B011C141A088312A800A90124
:10002800A900A801013083169B001C141A0883122A
:10003800A8070318A90A023083169B001C141A0883
:100048008312CD00033083169B001C141A088312F8
:10005800C100043083169B001C141A088312B000D8
:10006800B101B100B001053083169B001C141A08B9
:100078008312B0070318B10A063083169B001C14BC
:100088001A088312D100073083169B001C141A0823
:100098008312C500083083169B001C141A088312AB
:1000A800B200B301B300B201093083169B001C14DF
:1000B8001A088312B2070318B30A0A3083169B0082
:1000C8001C141A088312D2000B3083169B001C14D0
:1000D8001A088312C6000C3083169B001C141A08D9
:1000E8008312B400B501B500B4010D3083169B002E
:1000F8001C141A088312B4070318B50A0E308316A5
:100108009B001C141A088312D3000F3083169B001F
:100118001C141A088312C700103083169B001C1485
:100128001A088312B600B701B700B601113083165A
:100138009B001C141A088312B6070318B70A12305A
:1001480083169B001C141A088312D40013308316DC
:100158009B001C141A088312C800143083169B00D5
:100168001C141A088312B800B901B900B801153077
:1001780083169B001C141A088312B8070318B90ABF
:10018800163083169B001C141A088312D5001730EA
:1001980083169B001C141A088312C9001830831692
:1001A8009B001C141A088312BA00BB01BB00BA01D9
:1001B800193083169B001C141A088312BA070318F7
:1001C800BB0A1A3083169B001C141A088312D60027
:1001D8001B3083169B001C141A088312CA001C309B
:1001E80083169B001C141A088312BC00BD01BD00B5
:1001F800BC011D3083169B001C141A088312BC070F
:100208000318BD0A1E3083169B001C141A0883129B
:10021800D7001F3083169B001C141A088312CB00CA
:10022800203083169B001C141A088312BE00BF01DD
:10023800BF00BE01213083169B001C141A088312CC
:10024800BE070318BF0A223083169B001C141A0825
:100258008312D800233083169B001C141A088312BB
:10026800CC00243083169B001C141A088312AA00A1
:10027800AB01AB00AA01253083169B001C141A0899
:100288008312AA070318AB0A263083169B001C1496
:100298001A088312CE00273083169B001C141A08F4
:1002A8008312C200283083169B001C141A0883127C
:1002B800AC00AD01AD00AC01293083169B001C14C5
:1002C8001A088312AC070318AD0A2A3083169B005C
:1002D8001C141A088312CF002B3083169B001C14A1
:1002E8001A088312C3002C3083169B001C141A08AA
:1002F8008312AE00AF01AF00AE012D3083169B0014
:100308001C141A088312AE070318AF0A2E3083167E
:100318009B001C141A088312D0002F3083169B00F0
:100328001C141A088312C4004D1C9E29831203133F
:100338000515A129831203130511511CA72983123E
:1003480003138515AA29831203138511521CB0299A
:10035800831203138514B329831203138510531CC6
:10036800B929831203130514BC298312031305103A
:10037800541CC229831203138517C529831203133A
:100388008513551CCB29831203130517CE29831215
:1003980003130513561CD429831203138617D72970
:1003A800831203138613571CDD29831203130617C0
:1003B800E029831203130613581CE629831203133A
:1003C8008616E9298312031386124E1CEF2983121D
:1003D80003130616F2298312031306124F1CF82979
:1003E800831203130614FB29831203130610501CEF
:1003F800012A83120313861508008312031386113A
:100408000800FF30E200E3000130E2020030031C84
:10041800E303E302620A0319630A031D082A8B0136
:1004280010308316850006308600073083129F003F
:1004380085018601831681130B1781160116811514
:10044800FF30831281008B160B1119308316990027
:100458009030831298002430831698008C168312EB
:100468008C120D208B172308220421042004031961
:10047800412B2108E3002008E20029086306031D38
:10048800472A28086206031D562A043085064D08A7
:10049800023A0319542A4108082504308506562AC9
:1004A8004108082531086306031D5C2A30086206E6
:1004B800031D6B2A083085065108023A0319692A78
:1004C80045080825083085066B2A4508082533089D
:1004D8006306031D712A32086206031D802A023052
:1004E80085065208023A03197E2A46080825023072
:1004F8008506802A4608082535086306031D862ACE
:1005080034086206031D952A013085065308023A0D
:100518000319932A4708082501308506952A4708B4
:10052800082537086306031D9B2A36086206031D43
:10053800AA2A803085065408023A0319A82A4808CE
:10054800082580308506AA2A480808253908630640
:10055800031DB02A38086206031DBF2A40308506ED
:100568005508023A0319BD2A49080825403085066E
:10057800BF2A490808253B086306031DC52A3A080F
:100588006206031DD42A803086065608023A0319EB
:10059800D22A4A08082580308606D42A4A0808251F
:1005A8003D086306031DDA2A3C086206031DE92A92
:1005B800403086065708023A0319E72A4B080825EF
:1005C80040308606E92A4B0808253F086306031DC4
:1005D800EF2A3E086206031DFE2A203086065808C8
:1005E800023A0319FC2A4C08082520308606FE2A00
:1005F8004C0808252B086306031D042B2A086206ED
:10060800031D132B103086064E08023A0319112BCE
:100618004208082510308606132B420808252D08A5
:100628006306031D192B2C086206031D282B0130B5
:1006380086064F08023A0319262B4308082501307D
:100648008606282B430808252F086306031D2E2B32
:100658002E086206031D3D2B083086065008023A14
:1006680003193B2B44080825083086063D2B44080F
:100678000825A001A101A201A30131304002031CF9
:10068800372AC0018316A0018312E201E301831611
:100698009C184B2B8312620883169B0083126208F6
:1006A800A13E84008313000883169A0003108B1B55
:1006B80003148B131C1555309D00AA309D009C1403
:1006C8001C1103188B178312E20A0319E30A00307E
:1006D8006302303003196202031C4B2B0D20831672
:1006E800241C7A2B8312031305157D2B8312031305
:1006F80005118316281C842B831203138515872B59
:1007080083120313851183162C1C8E2B831203135B
:100718008514912B8312031385108316301C982B94
:100728008312031385149B2B8312031385108316DE
:10073800341CA22B831203138514A52B83120313D5
:1007480085108316381CAC2B831203138514AF2B2A
:1007580083120313851083163C1CB62B83120313D4
:100768000515B92B8312031305118316401CC02BE2
:10077800831203138515C32B831203138511831664
:10078800441CCA2B831203138514CD2B8312031325
:1007980085108316481CD42B831203138514D72B7A
:1007A80083120313851083164C1CDE2B831203134C
:1007B8008514E12B8312031385108316501CE82B34
:1007C800831203138514372A831203138510372ADB
:1007D80000308312031361246724031DFE2BF60ADD
:1007E8000319F70A02307702273003197602031833
:1007F8000800F02B003061246724031D0E2CF60A34
:100808000319F70A013077020F300319760203182B
:100818000800002C0030770287300319760203188D
:100828001E2C2708A3002608A2002508A1002408DA
:10083800A0000800F801203078020318582C003076
:1008480061246724031D332CF60A0319F70A0030C4
:10085800770229300319760203180800252C003086
:1008680061246724031D432CF60A0319F70A003094
:1008780077026F300319760203180800352C03102D
:10088800A00DA10DA20DA30D00307702243003198D
:100898007602031C562CA00A0319A10A0319A20AFE
:1008A8000319A30AF80A1F2C2308A7002208A60088
:1008B8002108A5002008A4000800051A0130F90045
:1008C800F601F70108000030051A01307906080022
:1008D80001300B1D00398B1E003900380319932C89
:1008E800EC230530302583122408F5002308F40092
:1008F800302583122308F5002208F40030258312DE
:100908002208F5002108F400302583122108F5009B
:100918002008F4003025FF30831281000B110130CC
:10092800831203138C1E003983168C1E003900387D
:100938000319D12C83128C128316A008031DA82C2E
:1009480083121A088316A0002008313A031DC02C10
:1009580031303025F401F50174089B001C141A0885
:100968003025F40A0319F50A0030750230300319EE
:100978007402031CB02CA0012008323A8312031D14
:10098800CD2C4008A03E84001A0883138000C00ABA
:100998008312981CD12C1812181673088A00720832
:1009A800840071088300FE0E7E0E0900DD01DE0161
:1009B800591CE42C5B08DD070318DE0A5C08DE0717
:1009C8000310DB0DDC0D0310DA0CD90C5A0859049E
:1009D800031DDC2C5E08DA005D08D900080004302D
:1009E800DB003E30FA000000FA0BF72C6400DB0B4A
:1009F800F52C0130D9020030031CDA03DA025A0858
:100A0800590403190800F32CDF00D900DA01E83093
:100A1800DB000330DC00DA245A08E1005908E00062
:100A28006108DA006008D900F32C763084007B3046
:100A3800282583132030840059302825A0308400CD
:100A4800D13028258301052A64008001840A040620
:100A5800031900340406292DF00070088312990048
:080A6800831698180800342DD4
:02400E00503F21
:10420000B0004F0000000100F0000F0000000500AA
:10421000D8002700000001003800C700000005009A
:10422000780087000000010060009F00000005008A
:10423000B800470000000100D0002F00000005007A
:104240005000AF000000010088007700000005006A
:10425000B0004F0000000100F0000F00000005005A
:00000001FF
